:1000000093C00000ACC00000AAC00000A8C000005F
:10001000A6C00000A4C00000A2C00000A0C0000054
:100020009EC000009CC00000C4C3000087C3000045
:1000300096C0000094C0000092C0000090C0000074
:100040008EC000008CC000008AC0000088C0000084
:1000500086C0000084C0000082C0000080C0000094
:100060007EC000007FC000007AC0000078C00000A1
:1000700076C0000074C0000072C0000070C00000B4
:100080006EC000006CC000006AC0000068C00000C4
:1000900066C0000064C0000062C0000060C00000D4
:1000A0005EC000005CC000005AC0000012011001D8
:1000B00002000008EB034B2001000102DC010902F1
:1000C0003E00020100C032090400000102020100EA
:1000D000052400100104240206052406000107057A
:1000E00082030800FF09040100020A00000007055E
:1000F0000402100001070583021000010403090433
:1001000018036200750073007700610072006500DB
:100110002E006400650000003003540043004D00D1
:10012000330031003000000011241FBECFEFDAE0B1
:10013000DEBFCDBF11E0A0E0B1E0EEEDF0E102C026
:1001400005900D92A632B107D9F712E0A6E2B1E010
:1001500001C01D92AA34B107E1F773D0BEC750CFDA
:10016000089508951F920F920FB60F9211242F93A6
:100170003F938F939F93CF93DF93EF93FF93909150
:10018000CE008EB38430D9F4C2EBD1E0E881F9819E
:100190009083888199810196998388832E813F81FC
:1001A0008217930721F48C819D81998388832FB7CF
:1001B000F8948A859B8501969B878A872FBFFF913C
:1001C000EF91DF91CF919F918F913F912F910F9060
:1001D0000FBE0F901F901895089580E091E0BDC666
:1001E00080E091E093C684B7877F84BF88E10FB633
:1001F000F89480936000109260000FBE80E090E061
:1002000020E80FB6F89420936100809361000FBE40
:100210006E9A769A729A6A98579A5F9A72D284E026
:1002200085BD80E190E09093CD008093CC0086E086
:100230008093CA0082E08093C80088E98093C90057
:1002400008952F923F924F925F926F927F928F927A
:100250009F92AF92BF92CF92DF92EF92FF920F9355
:100260001F93DF93CF93CDB7DEB72A970FB6F894DD
:10027000DEBF0FBECDBFDE011196EBE1F1E08AE0FB
:1002800001900D928150E1F7AEDFE6E2F1E02FB789
:10029000F89482E391E091838083938382839583B2
:1002A000848382EB91E09783868380E890E0918756
:1002B0008087138612862FBFE2EBF1E02FB7F89408
:1002C0008EEB91E0918380839383828395838483F3
:1002D0008EE392E09783868380E890E09187808721
:1002E000138612862FBF7894CC24DD24EE24FF24BD
:1002F00046E2A42E41E0B42E32EB232E31E0332E21
:100300002E010894411C511C2BE0622E712C6C0EA6
:100310007D1E98EC892E912CE114F10441F48EB3EA
:10032000843019F4769A5F9802C076985F9A8FB7F6
:10033000F89420913001309131018FBF80912E01CE
:1003400090912F012817390749F180E091E03BD5C2
:1003500097FD24C0F501AF010190F081E02D80836D
:10036000DA018D919C911197019611969C938E9331
:1003700016962D913C9117978217930731F4149696
:100380008D919C9115978D939C932FB7F894FA01BA
:10039000828593850196938782872FBF8FB7F894C4
:1003A0000091BC011091BD018FBFA89904C0093C08
:1003B000110508F45EC0A89A0894C11CD11CE11470
:1003C000F10461F4629B18C0F9EECF16F3E0DF068A
:1003D00008F44CC08EB3843079F448C0C6016AE793
:1003E00070E067D6892B21F48EB190E489278EB90D
:1003F00081E0E82EF12C3AC05F9B08C05F9886EF41
:1004000099E0F4013197F1F70197D9F7F201908162
:100410008091C80085FFFCCF9093CE003196E61501
:10042000F705A9F7E5CFE091B401F091B50180E0BF
:1004300091E0608146D58823E1F4F10182819381C6
:10044000019693838283268137818217930721F453
:1004500084819581938382832FB7F89482859385D5
:100460000197938782872FBF015010400115110516
:10047000D1F62FB7F89480913001909131012FBFC0
:10048000892B49F1F501AF010280F381E02D319113
:10049000DA011396FC93EE93129716968D919C9128
:1004A0001797E817F90741F414968D919C911597C9
:1004B00013969C938E9312972FB7F894FA01828526
:1004C00093850197938782872FBF8091C80085FF0E
:1004D000FCCF3093CE0080E091E0E4D460D41CCF18
:1004E000DA01923049F0933061F09130F9F4ECEA9E
:1004F000F0E022E130E01EC0EEEBF0E02EE330E071
:1005000019C0813049F0813018F0823079F408C088
:10051000ECEFF0E0849107C0E0E0F1E0849103C0EB
:10052000E8E1F1E08491282F30E004C0E0E0F0E061
:1005300020E030E0ED93FC93C90108958F70809323
:10054000E9008091EB0081608093EB001092ED0058
:100550006093EC004093ED008091EE00881F8827A7
:10056000881F08950F931F93CF93DF93062FEC01FD
:1005700010E02AC09881992329F16B81E981FA81E1
:100580002C81892F8F70873018F5223010F452E0BB
:1005900001C056E040E028E030E003C04F5F220F8A
:1005A000331F2E173F07D0F36295660F660F607CEE
:1005B000991F9927991F692B4295407F452BBEDFD4
:1005C000882331F01F5F25961017A0F281E001C04B
:1005D00080E0DF91CF911F910F91089580914202A9
:1005E00088238CF403C08EB38823B1F08091E80097
:1005F00082FFF9CF8091E8008B778093E80008951F
:100600008EB3882349F08091E80080FFF9CF809174
:10061000E8008E778093E80008954091E4005091BF
:10062000E50024E68091EC0080FF23C08091E80083
:1006300080FD1DC08EB3882311F482E008958530BB
:1006400011F483E008958091EB0085FF02C081E002
:1006500008958091E4009091E5008417950711F3C7
:10066000222311F484E008952150AC01DBCF80E017
:1006700008958091E80082FFDDCFF9CFEF92FF92DD
:100680000F931F934ED055D008ED10E0F8018081F4
:100690008F77808380818068808380818F7D808355
:1006A00019BC1EBA10923E021092400210923F02F4
:1006B00080EEE82EF12CF70180818B7F8083F8019A
:1006C00080818160808380E060E042E037DFE1EE9E
:1006D000F0E080818E7F8083E2EEF0E080818160B7
:1006E0008083808188608083F70180818E7F808312
:1006F000F8018081806180831F910F91FF90EF90BE
:100700000895E8EDF0E080818F7E8083E7EDF0E0F2
:1007100080818160808384E082BF81E08093410298
:10072000ADCFE8EDF0E080818E7F80831092E20013
:1007300008951092DA001092E10008951F920F922E
:100740000FB60F9211241F932F933F934F935F93F4
:100750006F937F938F939F93AF93BF93EF93FF9389
:100760001091E9008091EC001092E9008091F00076
:10077000877F8093F0007894A8D11092E90080914F
:10078000F00088608093F0001F701093E900FF91E3
:10079000EF91BF91AF919F918F917F916F915F91F9
:1007A0004F913F912F911F910F900FBE0F901F906F
:1007B00018951F920F920FB60F9211242F933F930B
:1007C0004F935F936F937F938F939F93AF93BF9359
:1007D000EF93FF938091E10082FF0AC08091E200D5
:1007E00082FF06C08091E1008B7F8093E100D6D22A
:1007F0008091DA0080FF1AC08091D80080FF16C077
:100800008091DA008E7F8093DA008091D90080FF9A
:100810000AC019BC82E089BD09B400FEFDCF81E0A9
:100820008EBB9EDC03C019BC1EBA9BDC8091E1002C
:1008300080FF17C08091E20080FF13C08091E2002A
:100840008E7F8093E2008091E20080618093E200DD
:100850008091D80080628093D80019BC85E08EBB5F
:100860009DD28091E10084FF2BC08091E20084FF43
:1008700027C019BC82E089BD09B400FEFDCF80917C
:10088000D8008F7D8093D8008091E1008F7E809387
:10089000E1008091E2008F7E8093E2008091E2008F
:1008A00081608093E20080913E02882331F4809140
:1008B000E30087FD02C081E001C084E08EBB6ED200
:1008C0008091E10083FF26C08091E20083FF22C077
:1008D0008091E100877F8093E10082E08EBB1092DF
:1008E0003E028091E1008E7F8093E1008091E200E2
:1008F0008E7F8093E2008091E20080618093E2002D
:1009000080E060E042E01ADE8091F0008860809331
:10091000F00044D2FF91EF91BF91AF919F918F91E1
:100920007F916F915F914F913F912F910F900FBEEB
:100930000F901F9018959C014091480250914902D8
:100940004617570718F4F90190E044C06115710586
:1009500011F0AB01F8CF8091E8008E778093E8002A
:1009600040E050E0F0CF8EB3882309F444C08530D6
:1009700009F443C08091E80083FF02C081E008953C
:100980008091E80082FD31C08091E80080FF22C0A4
:100990008091F3009091F200782F60E0292F30E0F1
:1009A000262B372B07C081918093F1004150504096
:1009B0002F5F3F4F4115510519F02830310598F34D
:1009C00090E02830310509F491E08091E8008E77BD
:1009D0008093E8004115510531F6992321F605C0B1
:1009E0008EB3882341F0853041F08091E80082FF8A
:1009F000F7CF80E0089582E0089583E008959C0198
:100A000040914802509149024617570718F4F901DE
:100A100090E045C06115710511F0AB01F8CF8091F0
:100A2000E8008E778093E80040E050E0F0CF8EB38E
:100A3000882309F446C0853009F445C08091E80058
:100A400083FF02C081E008958091E80082FD33C0F9
:100A50008091E80080FF23C08091F3009091F20024
:100A6000782F60E0292F30E0262B372B08C08491A7
:100A70008093F1003196415050402F5F3F4F411518
:100A8000510519F02830310590F390E028303105F8
:100A900009F491E08091E8008E778093E800411599
:100AA000510529F6992309F0C2CF05C08EB38823DA
:100AB00041F0853041F08091E80082FFF7CF80E07F
:100AC000089582E0089583E008950F931F93DF93C4
:100AD000CF93CDB7DEB7AC970FB6F894DEBF0FBE9D
:100AE000CDBFE2E4F2E08091F100819322E0EA34AC
:100AF000F207C9F772DB8091E80083FF36C180916D
:100B0000420230914302353009F487C0363040F458
:100B10003130C9F1313070F0333009F026C133C0C3
:100B2000383009F4F5C0393009F404C1363009F021
:100B30001CC196C0803821F0823809F016C108C067
:100B400090913F0280914002882399F0926011C0F9
:100B5000809146028F708093E9008091EB0090E0D5
:100B600025E0969587952A95E1F7982F9170109238
:100B7000E9008091E800877F8093E8009093F1007E
:100B80001092F100D0C0882319F0823009F0EDC036
:100B900090E08F719070009721F0029709F0E5C006
:100BA0000CC080914402813009F0DFC010924002F5
:100BB000333069F5809340022AC080914402882333
:100BC00031F5209146022F7009F4CFC02093E9003F
:100BD0008091EB0080FF1BC0333021F48091EB004B
:100BE000806213C08091EB0080618093EB0081E014
:100BF00090E002C0880F991F2A95E2F78093EA00DF
:100C00001092EA008091EB0088608093EB001092D4
:100C1000E9008091E800877F89C0882309F0A5C09A
:100C2000109144021F770FB7F8948091E800877FF6
:100C30008093E800D3DC8091E80080FFFCCF8091B6
:100C4000E3008078812B8093E30080688093E30049
:100C5000112311F482E001C083E08EBB0FBF85C079
:100C60008058823008F081C0809144029091450202
:100C700023E08C3D920709F033C083E08C838AE245
:100C80008B837FB7F894DE0115966EE040E050E06C
:100C900011E2E62FF0E010935700849140FF03C06B
:100CA00082958F706F5F8F70282F30E08A3018F038
:100CB000C901C79602C0C901C0968D939D934F5F2D
:100CC0005F4F4431510529F77FBF8091E800877F4E
:100CD0008093E800CE0103966AE270E02CDE12C039
:100CE00060914602AE014F5F5F4FFADBBC01009797
:100CF00009F43BC08091E800877F8093E8008981F8
:100D00009A817DDE8091E8008B778093E8002DC08A
:100D1000803859F58091E800877F8093E8008091C2
:100D20003E028093F1008091E8008E778093E80086
:100D300055DC1BC08823C9F4909144029230A8F47A
:100D40008091E800877F8093E80090933E0246DC24
:100D500080913E02882331F48091E30087FD02C038
:100D600081E001C084E08EBB3BDA8091E80083FF24
:100D70000AC08091EB0080628093EB008091E800D4
:100D8000877F8093E800AC960FB6F894DEBF0FBE65
:100D9000CDBFCF91DF911F910F91089508951F93BB
:100DA0008EB3882371F01091E9008091EC001092CD
:100DB000E9008091E80083FF01C087DE1F70109377
:100DC000E9001F910895FC018EB3843099F5848960
:100DD0009589A689B7890097A105B10559F1868142
:100DE0008F708093E9008091E80082FF23C04091DA
:100DF000F3002091F200942F80E030E0822B932BBF
:100E0000892B19F46FEF7FEF04C08091F100682FF8
:100E100070E04091F3002091F200942F80E030E0E8
:100E2000822B932B892B41F48091E8008B77809360
:100E3000E80002C06FEF7FEFCB0108950895FC0139
:100E40008EB3843051F584899589A689B789009736
:100E5000A105B10511F181818F708093E900409166
:100E6000F3002091F200942F80E030E0822B932B4E
:100E7000892BA9F09091E8008091E8008E7780930B
:100E8000E80095FD0CC0C9DB982F882349F48091B8
:100E9000E8008E778093E80003C092E001C090E004
:100EA000892F0895FC018EB3843051F4848995898B
:100EB000A689B7890097A105B10511F0CF01BFCF71
:100EC00008951F93FC01162F8EB38430E1F48489BA
:100ED0009589A689B7890097A105B105A1F08181FF
:100EE0008F708093E9008091E80085FD08C08091B3
:100EF000E8008E778093E80090DB882329F4109334
:100F0000F10080E001C082E01F910895CF93DF934C
:100F1000EC014096FC018BE0DF011D928A95E9F718
:100F200082E08C83898783E08E87CE01019661E021
:100F300019DB882371F0CE01069661E013DB88236C
:100F400041F0CE010B9661E00DDB882319F081E0C2
:100F500001C080E0DF91CF910895CF93DF93EC0142
:100F60008091E80083FFA2C0888190E02091460232
:100F7000309147022817390709F098C08091430241
:100F8000813269F0823220F4803209F08FC03CC097
:100F9000823209F46AC0833209F088C079C0809136
:100FA0004202813A09F082C08091E800877F8093F5
:100FB000E8008091E80080FFFCCF8C899D89AE8994
:100FC000BF898093F100292F3A2F4B2F552720936B
:100FD000F1009D01442755272093F1008B2F99277D
:100FE000AA27BB278093F100888D8093F100898D1B
:100FF0008093F1008A8D8093F1008091E8008E77D4
:101000008093E800EBDA52C080914202813209F00D
:101010004DC08091E800877F8093E80004C08EB3C4
:10102000882309F443C08091E80082FFF8CF8091C3
:10103000F1009091F1002091F1003091F1008C8B42
:101040009D8B2E8B3F8B8091F100888F8091F100DA
:10105000898F8091F1008A8F8091E8008B7780934F
:10106000E800BCDACE01B8D821C0809142028132BA
:10107000E9F48091E800877F8093E800AFDA8091FF
:10108000440290914502998B888BCE01D7DE0EC029
:1010900080914202813251F48091E800877F8093F1
:1010A000E8009CDACE0160914402C8DEDF91CF9166
:1010B0000895AA1BBB1B51E107C0AA1FBB1FA6179F
:1010C000B70710F0A61BB70B881F991F5A95A9F7F1
:0E10D00080959095BC01CD010895F894FFCF56
:1010DE0000831000000104100000018208000001CE
:1010EE000000000000000000000000550003000595
:0610FE00A6090101280013
:00000001FF
